:100000000C9434000C9400000C9400000C9400003C
:100010000C9400000C9400000C9400000C94000060
:100020000C9400000C9400000C9400000C94000050
:100030000C9400000C942D010C9400000C94000012
:100040000C9400000C9400000C94F3000C9402013A
:100050000C9413010C9400000C9400000C9400000C
:100060000C9400000C9400000FEF0DBF08E00EBFD1
:1000700099278FEF0E94DF000FE107B998B97894B4
:1000800002C0FFCFF894409AA0E0B1E01091C10007
:1000900010691093C100109103011330E1F7109122
:1000A000C1001F761093C1009093C6009093030186
:1000B0000E947B0060FDE7CF61FDE5CF62FD0E94FD
:1000C000930063FDE0CF64FDDECFA0E0B1E01091CE
:1000D000C10010621093C100109103011430E1F7C8
:1000E0001091C10017791093C1009093C6009093AE
:1000F0000301449AC8CF419A009100010F7061E05A
:10010000002319F0660F0A95FBCF772700910101B4
:100110000F70702B009102010F700295702B11F47B
:100120000C9443000895429A70930001709301016A
:1001300070930201A0E0B1E01091C1001062109331
:10014000C100109103011430E1F71091C10017793B
:100150001093C1009093C60090930301A0E0B2E019
:100160001091C10010691093C10010910301072F75
:10017000000F1017D1F71091C1001F761093C10026
:100180009093C60090930301439AA0E0B2E0C0E0D0
:10019000C395D2E0E0E0F2E00C911296188122962D
:1001A0000F701F701295012B01937A95A9F700E942
:1001B00000930001009301010093020108959093C0
:1001C000C6009093C0009093C1009093C20010E0CD
:1001D0001093C50013E31093C40016E01093C200FF
:1001E0009093030108951F935091C600152F107F1F
:1001F000103931F45D9310910301139510930301AD
:100200001F9118951F935D915093C60010910301A3
:100210001395109303011091C1001F7D1864109372
:10022000C1001F9118951F931091C100177B106298
:100230001093C1001F9118959093800090938100B6
:1002400090938200909385009093840090936F0028
:10025000909310019093110108953F9330911001F4
:10026000339520911201321719F43327809311012D
:08027000309310013F91189535
:00000001FF
